:1000000012C0189518951895189518951895189563
:100010008AC01895189518951895189518951895DB
:100020001895189518958FE58DBFC8E3E0E24E2E20
:1000300084E08EBFD4E0F4E05F2EA89584B7082E4C
:10004000877F84BF88E1992781BD91BDEEEFF3E002
:10005000A0E6B0E088278D933197E9F766248D9A62
:10006000959A82E0E0E3A7D3A0E6B0E0E5E7F0E010
:1000700098E039D4A09AA19AA298BDD2A89A8AE011
:1000800090E0CDD2A898A99818C05A924A9287E0D9
:10009000D2018C9381E0D2D25A924A9281E0D2016D
:1000A0008C9381E0CBD23FD1249682E087D2A8986E
:1000B00047D182E090E0B3D2A89A81EE80937F008E
:1000C0005A924A9281E0D2018C9381E0B7D222D138
:1000D000229681E073D287E280937F0080E3809351
:1000E00080005A924A9282E0D2018C9381E0A6D29B
:1000F00011D1229681E062D280E08FBD85E08EBD75
:1001000078947BB77F7B7BBF7BB77F777BBF79B7EB
:10011000746079BF85E08EBD06C075B77F7070686A
:1001200075BF8895FACF0F921F922F923F924F92F0
:100130005F927F92AF92BF920F931F932F933F9343
:100140004F935F936F937F938F939F93AF93BF93DF
:10015000CF93DF93EF93FF938FB78F9305D274D133
:1001600080EA80937F008AEA809380008BEB809303
:1001700081008CEC8093820080917E0080938300CC
:1001800080917D00809384005A924A9286E0D20149
:100190008C9381E053D2BED0229681E00FD282E0D0
:1001A00090E03DD2A89A81E090E039D2A89884E608
:1001B00090E035D280E090E0A2ECB0E08D939C938B
:1001C0009A9974C05A924A9287E0D2018C9381E046
:1001D00035D25A924A9281E0D2018C9381E02ED29C
:1001E000A2D0249682E0EAD10091A00040E7042347
:1001F000A1ECB0E00C930091C100003109F021C0E6
:1002000081EE80937F005A924A9281E0D2018C93D2
:1002100081E014D27FD0229681E0D0D187E2809312
:100220007F0080E1809380005A924A9282E0D2015E
:100230008C9381E003D26ED0229681E0BFD149C079
:1002400035C0003209F013C087E280937F0080E25E
:10025000809380005A924A9282E0D2018C9381E08E
:10026000EDD158D0229681E0A9D133C01FC081EED4
:1002700080937F005A924A9281E0D2018C9381E070
:10028000DDD148D0229681E099D187E280937F002A
:1002900080E3809380005A924A9282E0D2018C934C
:1002A00081E0CCD137D0229681E088D181E090E006
:1002B000B6D1A2ECB0E086D1A2ECB0E00D911C91D9
:1002C000043650E0150710F009F001C001C001C06C
:1002D00077CF959881E090E0A2D1959A8F918FBFCA
:1002E000FF91EF91DF91CF91BF91AF919F918F914E
:1002F0007F916F915F914F913F912F911F910F913E
:10030000BF90AF907F905F904F903F902F901F9045
:100310000F901895A998A881B9819C91AFE7B0E09A
:1003200063D1A99A0895A99891E0AA81BB815CD173
:10033000A881B9819C91A0EAB0E04ED1A99A089514
:100340008AE280937F0084E38093800083E480933B
:10035000810080E18093820080E18093830081E0CE
:10036000809384005A924A9286E0D2018C9381E075
:1003700065D1D0DF229681E021D181E280937F0098
:1003800081E0809380005A924A9282E0D2018C935D
:1003900081E054D1BFDF229681E010D182E28093C8
:1003A0007F0081E0809380005A924A9282E0D201DD
:1003B0008C9381E043D1AEDF229681E0FFD085E2CD
:1003C00080937F0088E2809380005A924A9282E074
:1003D000D2018C9381E032D19DDF229681E0EED074
:1003E00081E380937F0085E0809380005A924A9257
:1003F00082E0D2018C9381E021D18CDF229681E0D2
:10040000DDD086E280937F008FE0809380005A9257
:100410004A9282E0D2018C9381E010D17BDF229658
:1004200081E0CCD080E280937F008FE080938000D9
:100430005A924A9282E0D2018C9381E0FFD06ADF27
:10044000229681E0BBD0089580E380937F0084E30F
:100450008093800083E48093810080E18093820018
:1004600080E18093830081E0809384005A924A92D5
:1004700086E0D2018C9381E0E1D04CDF229681E0CE
:100480009DD08AE280937F0084E38093800083E4A0
:100490008093810080E18093820080E180938300DB
:1004A00081E0809384005A924A9286E0D2018C9334
:1004B00081E0C4D02FDF229681E080D081E280935A
:1004C0007F0081E0809380005A924A9282E0D201BC
:1004D0008C9381E0B3D01EDF229681E06FD082E260
:1004E00080937F0081E0809380005A924A9282E05C
:1004F000D2018C9381E0A2D00DDF229681E05ED004
:1005000085E280937F0088E2809380005A924A922D
:1005100082E0D2018C9381E091D0FCDE229681E0D2
:100520004DD086E280937F008FE0809380005A92C6
:100530004A9282E0D2018C9381E080D0EBDE229659
:1005400081E03CD080E280937F008EE08093800049
:100550005A924A9282E0D2018C9381E06FD0DADE27
:10056000229681E02BD0089582E0E0E382D05CEC1B
:1005700082E0E0E3A0D054E482E0E0E39CD080E2BB
:1005800093E04DD082E0E0E3A0E6B0E089D15EEBFD
:1005900082E0E0E390D082E0A8E6B0E0E0E329E08A
:1005A0002A93B1D08091680080937D00809169008A
:1005B00080937E000895481A590A0895481A88279A
:1005C000580A0895ED91FC91EF5FFF4FFC93EE9375
:1005D00008953197F1F7089515D08C9115D08D932A
:1005E0009A95D9F710D008950DD08D910DD09A9588
:1005F000E1F709D00895BD9ABC98C49ABB9A80E5EA
:100600008DB90895089508958FB9779BFECF8FB166
:100610000895689462F80895E89462F80895EF9355
:10062000FF93EE27E82BE92B31F0EAEFF0E031976A
:10063000F1F70197D1F7FF91EF910895480E8827C0
:10064000581E089591E0882321F08894991F8A9577
:10065000E9F7892F90950895883018F01196885001
:10066000FBCF08950181082B018312811923128386
:100670000895D2DFFF27E6DFF5DFEF93FF93E4E78E
:10068000F0E0A7DFFF91EF91182B1283092301837C
:10069000EF93FF93EEE0F0E09CDFFF91EF9110818C
:1006A000182309F0B6DFEF93FF93E3E6F0E091DF64
:1006B000FF91EF910895C6DFFF2721E048E005C0D4
:1006C000C1DFFF2729915D9148E0CCDF579510F4F9
:1006D000182B1283EF93FF93EAE0F0E07ADFFF91AB
:1006E000EF91182B128300000000000000000000B2
:1006F0000000000000000000000000004A9529F7FB
:100700002A9509F708959EDFFF27299148E055278C
:10071000A9DF0923018300000000000000000000A1
:1007200000000000000000000000889410811823E1
:1007300009F008945795EF93FF93EAE0F0E049DF62
:10074000FF91EF914A9521F75D932A95F9F6089567
:1007500089DF092301830000000000000000000081
:1007600000000000000000000000E8941081182341
:1007700009F06894EF93FF93EAE0F0E02ADFFF913D
:10078000EF9108956FDF16F4182B1283EF93FF9308
:10079000EAE0F0E01EDFFF91EF91182B12830000DA
:1007A0000000000000000000000000000000000049
:1007B00000000000089533273093740030937100D7
:1007C00058DF0EF458C03091710030FD54C06627D8
:1007D0006093730063956093720021E050EF48E0EE
:1007E00074DFB6DF31F9B4DF32F9632F667066303B
:1007F00009F441C0603019F031FB40D025C0609150
:100800007200709174006717B1F0C0F48F939F93DA
:10081000862F8A95A5E7B0E01FDF14DF7C9178234F
:100820006894772329F4E8946091720060937300D0
:100830009F918F9109C0689421D006C0E8941ED082
:1008400060917200609373009DDF60917200639508
:1008500060937200613409F0C4CF609173006093BB
:1008600074006623E89409F4689430F930937100B9
:10087000E89462F80895689462F808958F939F93BE
:10088000A5E7B0E0809172008A95E6DEDBDE7C9120
:1008900016F4782B01C079237C939F918F91089552
:1008A000AF93BF93EF93FF9338E0E5E7F0E00D914E
:1008B00001933A95E1F7FF91EF9130E430937400A2
:1008C0003327309371007CDF38E0BF91AF91E5E7CB
:1008D000F0E00D914191041719F43A95D1F708957C
:1008E00098DE089594E081918D939A95E1F70895AB
:00000001FF
